:100000000C94340018950000189500001895000015
:10001000189500001895000018950000189500002C
:10002000189500001895000018950000189500001C
:10003000189500000C94450E1895000018950000C6
:1000400018950000189500001895000018950000FC
:1000500018950000189500001895000018950000EC
:1000600018950000189500008FEF8DBFC0ECE8E9EF
:100070004E2E84E08EBFD4E0F4E05F2EEEEFF3E08E
:10008000A0E0B1E088278D933197E9F70E94201016
:10009000662481E080930001289A299A2A9A2B9A53
:1000A0002C9A81EE84B92D9A5E985F9880E08093B7
:1000B000800081E08093810078940C945401EAEDF3
:1000C000F0E080E40E946E1058E0C895802D0E94F8
:1000D000681031965A95C9F704C00000000000006E
:1000E000000FEEEFF0E088E40E946E1058E0C89533
:1000F000802D0E94681031965A95C9F704C00000FF
:10010000000000000F0FE2E2F1E080E50E946E10B7
:1001100058E0C895802D0E94681031965A95C9F70D
:1001200004C000000000000F0F0FE6E4F1E088E5D6
:100130000E946E1058E0C895802D0E94681031967C
:100140005A95C9F704C0000000000F0F0F0FEAE630
:10015000F1E080E60E946E1058E0C895802D0E9464
:10016000681031965A95C9F704C00000000F0F0FB0
:100170000F0FEEE8F1E088E60E946E1058E0C89597
:10018000802D0E94681031965A95C9F704C000006E
:100190000F0F0F0F0F0FE2EBF1E080E70E946E10E0
:1001A00058E0C895802D0E94681031965A95C9F77D
:1001B00004C0000F0F0F0F0F0F0FE6EDF1E088E7FF
:1001C0000E946E1058E0C895802D0E9468103196EC
:1001D0005A95C9F704C00F0F0F0F0F0F0F0F0E9492
:1001E0000B100895A2E0B1E00D911C91A4E0B1E0E4
:1001F0004D915C91040F151FA2E0B1E00D931C938B
:10020000A2E0B1E00D911C91A6E0B1E04D9155271F
:100210000E94C00FA2E0B1E04D935C938FEBA1E090
:10022000B1E01C910E941A10A2E0B1E00D911C9166
:10023000083050E015070CF402C00C943001A2E025
:10024000B1E08C910E9468108FE7A1E0B1E01C91B1
:100250000E941A10E0EDF2E20E9402100C944A0192
:1002600087E00E946810A2E0B1E00D911C9148E087
:1002700050E0041B150BA2E0B1E00D931C938FE737
:10028000A1E0B1E01C910E941A10A2E0B1E08C91B3
:100290000E946810A1E0B1E08C918F5F8C938FEB8E
:1002A00015E10E941A10089584E68093090180E800
:1002B0008093910180E8809393010C94960380E8E9
:1002C0008093910180E08093160181E08093170173
:1002D0008FEF80930901089580E88093930181E076
:1002E0008093160181E0809317018FEF80930901BD
:1002F000089500911601023011F00C94A701A2E9B3
:10030000B1E00D911C91A5E1B1E04D915527040F8D
:10031000151FA2E9B1E00D931C93A3E1B1E04D914B
:100320005C91A2E9B1E00D911C91041715071CF036
:1003300011F00C949D010C94A501A1E1B1E08D9107
:100340009C91A2E9B1E08D939C930C94E60101305D
:1003500011F00C94CC01A0E9B1E00E94AE0FAFE027
:10036000B1E04D915C91A0E9B1E00D911C910417B1
:1003700015071CF011F00C94BF010C94C701ADE0FF
:10038000B1E08D919C91A0E9B1E08D939C9380E8C0
:10039000809393010C94E601AAE0B1E08C918F5F09
:1003A0008C9340910C0100910A01041718F011F090
:1003B0000C94DC010C94E00180910B0180930A0104
:1003C00080E88093910180E88093930108950091E3
:1003D0001601023011F00C941302A2E9B1E00D9164
:1003E0001C91A5E1B1E04D915527041B150BA2E925
:1003F000B1E00D931C93A1E1B1E04D915C91A2E9B4
:10040000B1E00D911C91041715070CF402C00C9477
:100410001102A3E1B1E08D919C91A2E9B1E08D932D
:100420009C930C944D02013011F00C943602A0E91B
:10043000B1E00E94B40FADE0B1E04D915C91A0E954
:10044000B1E00D911C91041715070CF402C00C9437
:100450003102AFE0B1E08D919C91A0E9B1E08D93C4
:100460009C9380E8809393010C944D0280910A0143
:100470008A9580930A0140910B0100910A010417AB
:1004800010F00C94470280910C0180930A0180E8DF
:100490008093910180E88093930108950091160163
:1004A000023011F00C9458020E946C010C94670207
:1004B000013011F00C9460020E945F010C946702FD
:1004C00080910B0180930A0180E880939101089547
:1004D00000911601013011F00C947C0200919301FF
:1004E000003811F40C947A0282E0809316018FEFA9
:1004F000809307010C948C02003011F00C948C0254
:1005000000919101003811F40C948C0281E08093E9
:1005100016018FEF809307010895E6E3F5E080E48C
:100520000E946E1058E0C895802D0E946810319688
:100530005A95C9F704C0040E1F00001F0E040E9444
:100540000B108FE711E00E941A1000911601003085
:1005500011F00C94AE0280E00E9468108FEB11E065
:100560000E941A1000911601013011F00C94BB0288
:1005700080E00E94681000919301003811F40C94FF
:10058000CE028FEB1CE00E941A100091160102307F
:1005900011F00C94CE0280E00E94681008958091C2
:1005A00009018093080100910801003011F40C94B6
:1005B000FA0203B141EE042BA7E0B1E00C930091E5
:1005C00007010F3F11F00C94EA0289E180930901C1
:1005D0000C94FA0282E080930901809108018A95C7
:1005E000809308018AE090E00E949B100E94380FDF
:1005F0000C94D30282E0809308010091080100303E
:1006000011F40C941F0303B141EE042BA7E0B1E0F9
:100610000C93009107010F3F11F00C94120383E03B
:1006200080930801809108018A95809308018AE0EF
:1006300090E00E949B100E94380F0C94FD020895D8
:1006400084E18093080100910801003011F40C94BA
:10065000430303B141EE042BA7E0B1E00C930091FA
:1006600007010F3F11F40C94380384E180930801D3
:10067000809108018A958093080181E090E00E94B2
:100680009B100C942303089584E18093080100914A
:100690000801003011F40C94660303B141EE042B01
:1006A000A7E0B1E00C93009107010F3F11F00C940B
:1006B0005B030C946603809108018A95809308017E
:1006C00081E090E00E949B100C9447030895A3E101
:1006D000B1E04D915C91A2E9B1E00D911C9104173C
:1006E00015071CF011F00C9477030C947F03A3E121
:1006F000B1E08D919C91A2E9B1E08D939C93A1E131
:10070000B1E04D915C91A2E9B1E00D911C9104170B
:1007100015070CF402C00C949503A1E1B1E08D9192
:100720009C91A2E9B1E08D939C93089583E080931E
:100730007A0070917A00706870937A000E940B10B2
:100740000E942B0AEEEFF0E0BB27A0E10E945011BF
:1007500045E050E0040F151FABE3B1E00D931C938F
:10076000E2EDF2E20E9402100E949E090E94440300
:10077000009107010F3F11F40C94C0030C94CE03B9
:10078000ABE3B1E04D915C91ACE2B1E00D911C9115
:10079000041715071CF011F00C94B40381E080934A
:1007A000840080E08093850080916F008160809359
:1007B0006F0081E080930A010E94380F0E941209A5
:1007C0000E94CF02009107010D3F11F00C94EA0343
:1007D0000E944E02009107010B3F11F00C94F203AE
:1007E0000E946802009107010F3E11F00C94FA0379
:1007F0000E94E70100910701073F11F00C940204E9
:100800000E9479010C94DE03E0EEF2E20E940210F5
:10081000009107010B3F11F40C9410040C94520446
:1008200084E690E0A4E0B1E08D939C938DE080930A
:1008300006010E945F000E94290BA3E2B1E08D91A6
:100840009C91AAE2B1E08D939C93ADE1B1E08D91D2
:100850009C91ACE2B1E08D939C93AFE1B1E08D91BE
:100860009C91AEE2B1E08D939C93A5E2B1E08D91B5
:100870009C91A0E3B1E08D939C93A1E2B1E08D91B6
:100880009C91A2E3B1E08D939C930E94DB090E94AE
:100890004403009107010D3F11F00C941B0481E00B
:1008A000809317010895E8EEF2E20E940210009191
:1008B00007010B3F11F40C945F040C94B10580E028
:1008C00090E0A4E0B1E08D939C9380E480930601D6
:1008D0000E945F00E4EFF2E20E9402100E94091001
:1008E000E4E0F3E20E94021080ED97E00E949B108A
:1008F00080ED97E0ADE3B1E08D939C9380E090E0D4
:10090000AFE3B1E08D939C9380ED97E0A1E4B1E07B
:100910008D939C9380E090E0A3E4B1E08D939C9351
:1009200080ED97E0A5E4B1E08D939C9380E090E0AA
:10093000A7E4B1E08D939C9380ED97E0A9E4B1E04A
:100940008D939C9380E090E0ABE4B1E08D939C9319
:100950000E940B100E949E09ADE3B1E04D915C91A5
:10096000AAE2B1E00D911C91041715070CF402C026
:100970000C94C204AAE2B1E08D919C91ADE3B1E088
:100980008D939C93AFE3B1E04D915C91AAE2B1E00D
:100990000D911C91041715071CF011F00C94D20452
:1009A0000C94DA04AAE2B1E08D919C91AFE3B1E03E
:1009B0008D939C93A1E4B1E04D915C91ACE2B1E0E8
:1009C0000D911C91041715070CF402C00C94F0044F
:1009D000ACE2B1E08D919C91A1E4B1E08D939C9348
:1009E000A3E4B1E04D915C91ACE2B1E00D911C91BA
:1009F000041715071CF011F00C9400050C94080561
:100A0000ACE2B1E08D919C91A3E4B1E08D939C9315
:100A1000A5E4B1E04D915C91AEE2B1E00D911C9185
:100A2000041715070CF402C00C941E05AEE2B1E0E9
:100A30008D919C91A5E4B1E08D939C93A7E4B1E0E6
:100A40004D915C91AEE2B1E00D911C910417150738
:100A50001CF011F00C942E050C943605AEE2B1E0BA
:100A60008D919C91A7E4B1E08D939C93A9E4B1E0B2
:100A70004D915C91A0E3B1E00D911C910417150715
:100A80000CF402C00C944C05A0E3B1E08D919C9154
:100A9000A9E4B1E08D939C93ABE4B1E04D915C91FE
:100AA000A0E3B1E00D911C91041715071CF011F0A3
:100AB0000C945C050C946405A0E3B1E08D919C91CD
:100AC000ABE4B1E08D939C930E94DB090E94440348
:100AD000009107010B3F11F00C94A805EAEFF0E03C
:100AE000ADE3B1E07BE70E943F11ECEFF0E0AFE354
:100AF000B1E07BE70E943F11EEEFF0E0A1E4B1E04E
:100B00007BE70E943F11E0E0F1E0A3E4B1E07BE786
:100B10000E943F11E2E0F1E0A5E4B1E07BE70E9432
:100B20003F11E4E0F1E0A7E4B1E07BE70E943F1170
:100B3000E6E0F1E0A9E4B1E07BE70E943F11E8E0E4
:100B4000F1E0ABE4B1E07BE70E943F110C94AE050D
:100B5000009107010D3F11F00C94AA0481E08093ED
:100B6000170108950895089500914D014AE00E94EB
:100B70005811AEE4B1E00C93A0E8B4E0EEE4F1E08B
:100B80000E94ED100E94FA0FE2E1F3E20E940210CF
:100B900000914D014AE00E945811AEE4B1E08C93FF
:100BA000A0E8B4E0EEE4F1E00E94ED100E94FA0F3C
:100BB000089500910A01013011F40C94E1050C94A0
:100BC000430600910701093F11F00C940206E4E18D
:100BD000F3E20E940210E0E0F0E0A0E5B1E091E075
:100BE0000E9451110E940910E4E2F3E20E940210F7
:100BF000A0E8B4E0E0E5F1E00E94ED100E94FA0FF9
:100C00000C9443068FE712E00E941A108091340181
:100C100080934D010E94B405ECE2F3E20E940210C1
:100C20008FE719E00E941A10A0E8B4E0EAE1F1E0D1
:100C30000E94ED100E94FA0F8091190180934F01DC
:100C40000E9444068091180180934F010E9444063F
:100C50008FEB12E00E941A10EBE0F1E0A8E3B1E0A4
:100C60000E944E110E94540A009107010B3F11F09F
:100C70000C94430680E08093180180E08093190172
:100C800080E080931A010895E2E3F3E20E940210EB
:100C900000914F010A3010F00C945206E4E3F3E2A5
:100CA0000E940210A0E8B4E0EFE4F1E00E94ED1031
:100CB0000E94FA0F0895E6E3F3E20E940210009109
:100CC0009101003811F00C947A06EBE0F1E0A0E914
:100CD000B1E00E944E1180E08093910180E090E0AD
:100CE000ADE0B1E08D939C9387E090E0AFE0B1E0A0
:100CF0008D939C938FEB12E00E941A1080919001CB
:100D0000809338010E94540A009107010B3F11F0B3
:100D10000C949506EBE0F1E0A0E9B1E07BE70E94DE
:100D20003D110E942B0A0E945F010895E4E4F3E262
:100D30000E94021000919101003811F00C94C70636
:100D400080E390E0ADE0B1E08D939C938FE790E07D
:100D5000AFE0B1E08D939C93A6E3B1E00D91112734
:100D600040E050E0040F151FA4E5B1E00D931C9383
:100D7000A4E5B1E0ED91FC91A0E9B1E091E00E9421
:100D8000511180E08093910180E0809353010091A4
:100D900007010B3F11F00C94F306A4E5B1E0ED91CF
:100DA000FC91A0E9B1E091E07BE70E944011A3E54E
:100DB000B1E08C918F5F8C9300915301083010F457
:100DC0000C94E6060E945F010C943107A4E5B1E0A3
:100DD0000E94AE0FA4E5B1E0ED91FC91A0E9B1E075
:100DE00091E00E9451118FEB12E00E941A10EBE08B
:100DF000F1E0A8E3B1E00E944E110E94540A02E023
:100E000040915301040FABE1B1E00C93ABE1B1E0D1
:100E10008C918E5F8C938FEBABE1B1E01C910E94C3
:100E20001A1000919001003411F00C941D07E0EDB0
:100E3000F2E20E9402100C942207A0E9B1E08C912A
:100E40000E94681000911601013011F00C943107D6
:100E50008FEBABE1B1E01C910E941A1080E080930F
:100E60001C010895E2E5F3E20E9402100091910155
:100E7000003811F00C94600780E090E0ADE0B1E044
:100E80008D939C9382E090E0AFE0B1E08D939C93D2
:100E9000A6E3B1E00D9111274DE150E0040F151FBD
:100EA000A6E5B1E00D931C93A6E5B1E0ED91FC91B0
:100EB000A0E9B1E091E00E94511180E0809391019E
:100EC0008FEB12E00E941A1000919001013011F096
:100ED0000C947007EAE5F3E20E9402100C947E077E
:100EE000023011F00C947A07E0E6F3E20E9402105F
:100EF0000C947E07E8E6F3E20E94021000910701DD
:100F00000B3F11F00C949007A6E5B1E0ED91FC9138
:100F1000A0E9B1E091E07BE70E9440110E945F01EF
:100F2000089500919101003811F00C94AC0781E014
:100F300090E0ADE0B1E08D939C9385E090E0AFE070
:100F4000B1E08D939C9381E090E0A0E9B1E08D93B6
:100F50009C9381E08093150100911601013010F0FF
:100F60000C94D30780913701809327010E940910C8
:100F700081E0809328010E94870883E08093280104
:100F80000E94870882E0809328010E94870880E001
:100F9000809328010E94870884E0809328010C94A4
:100FA00087080C9486088CE99FEFA1E1B1E08D934E
:100FB0009C9384E690E0A3E1B1E08D939C938FEB4A
:100FC00012E00E941A1000919001013011F00C946F
:100FD0001E08E4E7F3E20E94021080E090E0A1E145
:100FE000B1E08D939C9381E090E0A3E1B1E08D931B
:100FF0009C935A924A9280E0A42DB52D8C9381E067
:101000000E94AA0F0E94D90A229681E00E94A60F90
:101010008FEB1DE00E941A1000919201003011F038
:101020000C941808EEE7F3E20E9402100C941C08DE
:10103000E2E8F3E20E9402100C948608023011F0FC
:101040000C943708E6E8F3E20E9402105A924A92A2
:1010500083E0A42DB52D8C9381E00E94AA0F0E94FD
:10106000D90A229681E00E94A60F0C9486080330CC
:1010700011F00C945008ECE8F3E20E9402105A922E
:101080004A9281E0A42DB52D8C9381E00E94AA0F95
:101090000E94D90A229681E00E94A60F0C9486082D
:1010A000043011F00C946908E4E9F3E20E940210A4
:1010B0005A924A9282E0A42DB52D8C9381E00E9431
:1010C000AA0F0E94D90A229681E00E94A60F0C94D2
:1010D0008608053011F00C948608EEE9F3E20E94D0
:1010E000021080E090E0A1E1B1E08D939C935A92D0
:1010F0004A9284E0A42DB52D8C9381E00E94AA0F22
:101100000E94D90A229681E00E94A60F08950E94AB
:10111000B00AA0E8B4E0E5E9F1E00E94E6100E9420
:10112000FA0FEAEAF3E20E9402100895ECEAF3E211
:101130000E94021000919101003811F00C94B20845
:1011400081E090E0ADE0B1E08D939C9383E090E08E
:10115000AFE0B1E08D939C9381E090E0A0E9B1E035
:101160008D939C9300911601013010F00C94BA08F5
:101170000C9411098FEB12E00E941A10009190015B
:10118000013011F00C94C8080E9404040C94110959
:10119000023011F00C94D0080E9453040C941109F1
:1011A000033011F00C941109E4EBF3E20E940210F9
:1011B00000919301003811F00C94F80880E090E061
:1011C000A1E1B1E08D939C9388EC90E0A3E1B1E0C4
:1011D0008D939C9381E080931501E9EFF0E0A2E903
:1011E000B1E00E944E1180E0809393010E9467035A
:1011F0008FEB1DE00E941A108091920180934D01A7
:101200000E94B405009107010B3F11F00C941109E5
:10121000E9EFF0E0A2E9B1E07BE70E943D110E9416
:101220006C01089581E080930B0189E080930C01AB
:1012300081E080931C010E948D028FE712E00E94E2
:101240001A1000910A01013011F00C942B090E9430
:10125000D9050C948509023011F00C9433090E94D1
:101260005B060C948509033011F00C944209E0EC04
:10127000F3E20E94021089E0809337010E949107F7
:101280000C948509043011F00C945109E6ECF3E25A
:101290000E9402108EE0809337010E9491070C9407
:1012A0008509053011F00C946009E0EDF3E20E942D
:1012B000021083E1809337010E9491070C94850905
:1012C000063011F00C946F09EAEDF3E20E9402106F
:1012D00088E1809337010E9491070C9485090730BB
:1012E00011F00C9477090E9432070C94850908309C
:1012F00011F00C947F090E9496060C948509093020
:1013000011F00C9485090E94960800911701003095
:1013100011F40C94930980E0809317018FEF809370
:1013200007010C94180900911C01003011F40C9471
:101330009D098FE715E10E941A10089580E08093BF
:101340007C000E94B410AAE2B1E08D939C9381E0EE
:1013500080937C000E94B410ACE2B1E08D939C932A
:1013600082E080937C000E94B410AEE2B1E08D93E5
:101370009C9383E080937C000E94B410A0E3B1E0D2
:101380008D939C9384E080937C000E94B410A2E330
:10139000B1E08D939C9385E080937C000E94B41013
:1013A000082F192F44E050E00E94C00FA4E3B1E0E1
:1013B0004D935C9308958CE00E946E1082E08093C0
:1013C0000101AEE2B1E08D919C91A2E0B1E08D937C
:1013D0009C930E94F200A1E0B1E08C918F5F8C930E
:1013E000AAE2B1E08D919C91A2E0B1E08D939C9333
:1013F0000E94F200A1E0B1E08C918F5F8C93A0E39A
:10140000B1E08D919C91A2E0B1E08D939C930E94FC
:10141000F200A1E0B1E08C918F5F8C93ACE2B1E07F
:101420008D919C91A2E0B1E08D939C930E94F2007B
:10143000A1E0B1E08C918F5F8C93A2E3B1E08D913C
:101440009C91A2E0B1E08D939C930E94F2008EE00B
:101450000E946E100895EBE0F1E0BB27A0E10E942E
:101460004E11083010F40C943E0AEBE0F1E0A0E1DC
:10147000BB2780E08C937BE70E943D11EBE0F1E01D
:10148000AAE5B1E00E944E11AAE5B1E00C914FE14E
:10149000049F0C92AAE5B1E08C918F5F8C938091B0
:1014A0005A01809336010895A8E3B1E08C918F5FD3
:1014B0008C93A0E8B4E0E8E3F1E00E94ED100E9414
:1014C000FA0FE2E3F3E20E940210809138018A955C
:1014D00080933801A8E3B1E00D9111274FE150E06E
:1014E0000E94AA10ABE5B1E00D931C93ABE5B1E00F
:1014F0000D911C9140E050E0040F151FABE5B1E0E9
:101500000D931C9381E080931B0100911B01083017
:1015100018F011F00C94AF0AABE5B1E00E94AE0FE9
:10152000ABE5B1E0ED91FC91ADE5B1E091E00E9459
:10153000511100915D01003411F00C94A20A80E277
:1015400080935D01ADE5B1E08C910E946810ABE144
:10155000B1E08C918F5F8C9311F00C94850A089503
:101560000091270140913601040FA9E2B1E00C93EC
:101570000091290140912801040FA9E2B1E00C93E8
:10158000A9E2B1E0EC91FF27A5E9B1E091E00E946A
:10159000511180E080939601009195010F3718F06A
:1015A00011F00C94D50A0C94D80A8FEF8093960111
:1015B000089500919301003811F00C940A0B0091EA
:1015C000360140913701040FAEE5B1E00C93009174
:1015D0005E01A881B9814C91040FAEE5B1E00C9396
:1015E000AEE5B1E0EC91FF27A2E9B1E091E00E9405
:1015F000511180E080939301009192010F3718F010
:1016000011F00C94050B0C94080B8FEF8093930151
:101610000E9467038FEB1DE00E941A10A0E8B4E05F
:10162000E2E9F1E00E94E6100E94FA0F0091070142
:101630000B3F11F00C94280BAEE5B1E0EC91FF27C5
:10164000A2E9B1E091E07BE70E9440110E946C01A9
:1016500008950E949E09ACE2B1E08D919C91A1E7B2
:10166000B1E08D939C93EEEFF0E0ACE7B1E00E9427
:101670005011E0E0F1E0AEE7B1E00E94501188E1E6
:1016800080937B010E94B20BA1E7B1E08D919C9108
:10169000AFE5B1E08D939C93AAE2B1E08D919C916E
:1016A000A1E7B1E08D939C93EAEFF0E0ACE7B1E005
:1016B0000E945011ECEFF0E0AEE7B1E00E94501153
:1016C0008EE080937B010E94B20BA1E7B1E08D9187
:1016D0009C91A1E6B1E08D939C93AEE2B1E08D9137
:1016E0009C91A1E7B1E08D939C93E2E0F1E0ACE73F
:1016F000B1E00E945011E4E0F1E0AEE7B1E00E94F9
:10170000501189E080937B010E94B20BA1E7B1E008
:101710008D919C91A5E6B1E08D939C93A0E3B1E0FF
:101720008D919C91A1E7B1E08D939C93E6E0F1E06F
:10173000ACE7B1E00E945011E8E0F1E0AEE7B1E0C3
:101740000E94501183E180937B010E94B20BA1E7BC
:10175000B1E08D919C91A3E6B1E08D939C930E94A2
:10176000480D0895AEE7B1E04D915C91ACE7B1E072
:101770000D911C91041715070CF002C00C94CC0BB2
:10178000AEE7B1E00D911C9142E050E0041B150B57
:10179000ACE7B1E00D931C93ACE7B1E04D915C91E7
:1017A000A1E7B1E00D911C91041715070CF402C0DC
:1017B0000C94E20BACE7B1E08D919C91A1E7B1E014
:1017C0008D939C93AEE7B1E04D915C91A1E7B1E0C0
:1017D0000D911C91041715071CF011F00C94F20BDD
:1017E0000C94FA0BAEE7B1E08D919C91A1E7B1E0CA
:1017F0008D939C93AEE7B1E00D911C91ACE7B1E005
:101800004D915C91041B150BA0E8B1E00D931C9366
:10181000A0E8B1E00D911C9142E050E00E94C00FA1
:10182000A0E8B1E04D935C93A1E7B1E00D911C916C
:10183000ACE7B1E04D915C91041B150BA1E7B1E061
:101840000D931C93A1E7B1E00D911C91A0E8B1E0CC
:101850004D915C91041B150BA1E7B1E00D931C9316
:10186000A1E7B1E00D911C9142E350E00E94AA1063
:10187000A1E7B1E00D931C93A0E8B1E00D911C919C
:1018800042E050E00E94C00FA0E8B1E04D935C93AD
:10189000A1E7B1E00D911C91A0E8B1E04D915C9100
:1018A0000E94C00FA1E7B1E04D935C9380917B0152
:1018B0008093270184E0809328010E94B00AA1E769
:1018C000B1E00D911C91A5E9B1E04D915C910E94B0
:1018D000AA10A7E7B1E00D931C93A7E7B1E00D9123
:1018E0001C9144E650E00E94C00FA7E7B1E04D9381
:1018F0005C93A1E7B1E00D911C91A7E7B1E04D9198
:101900005C91041B150BA9E7B1E00D931C93A5E9AD
:10191000B1E00D911C91A1E7B1E04D915C910E9465
:10192000AA10A7E7B1E00D931C93A7E7B1E00D91D2
:101930001C9144E650E00E94C00FA7E7B1E04D9330
:101940005C930E942D0D0E942D0DA9E7B1E00D9131
:101950001C91A7E7B1E04D915C91040F151FA1E721
:10196000B1E00D931C9383E0809328010E94B00A9C
:10197000A5E9B1E08D919C91A2E8B1E08D939C9393
:10198000A1E7B1E00D911C91003050E015071CF06B
:1019900011F00C94CD0C0C94F20C82E08093280191
:1019A0000E94B00AA5E9B1E00D911C91A2E8B1E056
:1019B0004D915C91041B150BA7E7B1E00D931C93AF
:1019C0000E942D0DA7E7B1E00D911C91A2E8B1E0B6
:1019D0004D915C91040F151FA1E7B1E00D931C938D
:1019E0000C94150D81E0809328010E94B00AA5E9AE
:1019F000B1E00D911C91A2E8B1E04D915C91041B06
:101A0000150BA7E7B1E00D931C930E942D0DA2E8E2
:101A1000B1E00D911C91A7E7B1E04D915C91041BE1
:101A2000150BA1E7B1E00D931C9380E08093280192
:101A30000E94B00A00919501003011F40C942C0D15
:101A4000A1E7B1E00D911C914FEF5FEF0E94AA104A
:101A5000A1E7B1E00D931C930895A7E7B1E00D91C4
:101A60001C91A1E7B1E04D915C910E94AA10A7E7FB
:101A7000B1E00D931C93A7E7B1E00D911C9144E6F2
:101A800050E00E94C00FA7E7B1E04D935C9308952A
:101A9000A1E6B1E08D919C91A3E2B1E08D939C937E
:101AA000A5E6B1E08D919C91AFE1B1E08D939C935F
:101AB000A5E6B1E08D919C91A1E2B1E08D939C935C
:101AC000A3E6B1E08D919C91A5E2B1E08D939C934A
:101AD000AFE5B1E08D919C91ADE1B1E08D939C9328
:101AE000A6E3B1E00D9111274DE150E0040F151F61
:101AF000A4E8B1E00D931C93A4E8B1E0ED91FC9152
:101B0000A5E9B1E091E00E945111009195010130E9
:101B100011F00C94CF0DA5E6B1E00D911C9142E0BF
:101B200050E00E94C00FA5E6B1E04D935C93A3E6A0
:101B3000B1E00D911C9142E050E00E94C00FA3E67D
:101B4000B1E04D935C93A5E6B1E00D911C91A3E645
:101B5000B1E04D915C91040F151FAFE1B1E00D9321
:101B60001C93A5E6B1E00D911C91A3E6B1E04D9167
:101B70005C91041B150BA1E2B1E00D931C93A5E64B
:101B8000B1E00D911C91A3E6B1E04D915C91041B75
:101B9000150BA5E2B1E00D931C930C94070E0230D7
:101BA00011F00C94070EA1E6B1E00D911C9142E0FA
:101BB00050E00E94C00FA1E6B1E04D935C93A3E614
:101BC000B1E00D911C9142E050E00E94C00FA3E6ED
:101BD000B1E04D935C93A1E6B1E00D911C91A3E6B9
:101BE000B1E04D915C91040F151FA3E2B1E00D939C
:101BF0001C93A1E6B1E00D911C91A3E6B1E04D91DB
:101C00005C91041B150BA5E2B1E00D931C93ADE1B3
:101C1000B1E00D911C9145E050E00E94AA10AFE6A2
:101C2000B1E00D931C93AFE1B1E00D911C9145E043
:101C300050E00E94AA10A7E6B1E00D931C93A1E228
:101C4000B1E00D911C9145E050E00E94AA10A9E678
:101C5000B1E00D931C93A5E2B1E00D911C9145E01C
:101C600050E00E94AA10ADE6B1E00D931C93A3E2F0
:101C7000B1E00D911C9145E050E00E94AA10ABE646
:101C8000B1E00D931C93089508950F921F922F9227
:101C90003F924F925F927F92AF92BF920F931F93AA
:101CA0002F933F934F935F936F937F938F939F9364
:101CB000AF93BF93CF93DF93EF93FF938FB78F9340
:101CC0002D9AEAE8FEE0EF93FF93E0E7FEE0A0E064
:101CD000B1E08C919927880F991FE80FF91F09949B
:101CE0000C94260F0C94260F0C94DB0E0C94260FEC
:101CF0000C94E80E0C94260F0C94F50E0C94260F01
:101D00000C94020F0C94260F0C940F0F0C94260FBA
:101D10000C941C0F0FEF1FEFA6E8B1E04D915C9102
:101D2000041B150BBB27A0E18D919C91909385001E
:101D300080938400A0E0B1E08C918F5F8C93A6E843
:101D4000B1E00D911C9144EB50E0040F151FA6E883
:101D5000B1E00D931C93A8E8B1E00D911D912D9178
:101D60003C91A6E8B1E04D915C91662777270E94EF
:101D7000C610A8E8B1E00D931D932D933D938F916C
:101D80008FBFFF91EF91DF91CF91BF91AF919F9165
:101D90008F917F916F915F914F913F912F911F9103
:101DA0000F91BF90AF907F905F904F903F902F909A
:101DB0001F900F90189508EE13E0A7E6B1E04D9143
:101DC0005C91040F151FA6E8B1E00D931C930895D4
:101DD00008EE13E0ABE6B1E04D915C91040F151FE6
:101DE000A6E8B1E00D931C93089508EE13E0ADE66C
:101DF000B1E04D915C91040F151FA6E8B1E00D9381
:101E00001C93089508EE13E0AFE6B1E04D915C91AC
:101E1000040F151FA6E8B1E00D931C93089508EE7A
:101E200013E0A9E6B1E04D915C91040F151FA6E8FF
:101E3000B1E00D931C93089580E797E1A6E8B1E027
:101E40008D939C9380E08093000108952D988CE2FF
:101E500091E0A6E8B1E08D939C93009100010730DA
:101E600011F00C94360F5F9A0C94370F5F98089519
:101E70000E94290B40E452E46FE070E0A8E8B1E072
:101E80000D911D912D913C910E94CB101CF011F0F1
:101E90000C944C0F0C94850FA8E1B1E08C918F5FEE
:101EA0008C9300E010E020E030E0A8E8B1E00D9372
:101EB0001D932D933C93009118010B3318F011F0F2
:101EC0000C94640F0C947D0F80E080931801A9E1BD
:101ED000B1E08C918F5F8C93009119010B3318F056
:101EE00011F00C94750F0C947D0F80E08093190114
:101EF000AAE1B1E08C918F5F8C930E94D905E9EF44
:101F0000F0E0ACE8B1E00E944E11289AACE8B1E0F4
:101F10004D915527A4E3B1E00D911C9104171507CD
:101F20000CF402C00C94A50F40EE53E964E070E09D
:101F3000A8E8B1E00D911D912D913C910E94CB102C
:101F40000CF402C00C94A50F28980895481A88270D
:101F5000580A0895480E8827581E0895ED91FC915F
:101F60003196FC93EE930895ED91FC913197FC939B
:101F7000EE93089509D00E94AA1000FC10D0089595
:101F800003D01ED001F8F9CF0024E89457FF02C017
:101F900009D0689400F80BD010F80124089502D0FD
:101FA00009D00895509540954F5F5F4F0895E8948C
:101FB00017FF0895009510950F5F1F4F68940895BF
:101FC000352F242FE894452B11F468940895512F50
:101FD000402F0027112780E1440F551F001F111FBC
:101FE000021B130B416018F4020F131F4E7F8A95DA
:101FF00099F70895A0E8B4E08D91882311F068D096
:10200000FBCF08950E94C210802D11F061D0FACF4D
:10201000089580EC63C081E061D00FD080E85EC09D
:102020008FE7213039F08FEB223021F08FE8233019
:1020300009F08FEC810F0C946E1083E099277BC020
:102040008AEF90E00E949B10539A529A519A509AAC
:10205000559A549A5C9885E090E00E949B105D9898
:102060005B985A98599A589A5D9AEF93FF93E5E1D5
:10207000F0E00E948F10FF91EF915D9859D05D9A2A
:10208000EF93FF93E5E1F0E00E948F10FF91EF9155
:102090005D984ED05D9AEF93FF93E5E1F0E00E94EA
:1020A0008F10FF91EF915D9843D058985D9AEF9310
:1020B000FF93E5E1F0E00E948F10FF91EF915D98B2
:1020C00037D088E20BD08EE009D086E007D00895A3
:1020D0005C9A829505D004D02BD008955C98F9CFF6
:1020E000859510F4589A01C05898859510F4599A1E
:1020F00001C05998859510F45A9A01C05A9885954F
:1021000010F45B9A01C05B985D9AEF93FF93E5E151
:10211000F0E00E948F10FF91EF915D980895319744
:10212000F1F70895689462F80895E89462F80895C4
:1021300081E090E000C0EF93FF93EE27E82BE92BBE
:1021400031F0EAEFF0E03197F1F70197D1F7FF9125
:10215000EF9108950F92B801469F8001479F100D9F
:10216000569F100D0F90089580917A00806C809397
:102170007A0080917A0086FDFCCF80917800909162
:1021800079000895C895319600200895040F151F11
:10219000261F371F089504171507260737070895C8
:1021A000000F111F221F331F0895009510952095D1
:1021B00030950F5F1F4F2F4F3F4F089501911081B2
:1021C0000EC001911191219130810BC001911081BC
:1021D00017FF05C03FEF2FEF04C000811127222712
:1021E000332737FF03C0E1DF8DE28D93CF93DF9379
:1021F000CF92DF92EF92AA24BB24CC24DD24EE24DC
:1022000040E2CAE0DD2755E093E38881890F87FD2E
:102210009F7083FD907F891B89935A95A9F7C0DF32
:10222000AA1CBB1CCC1CDD1CEE1C4A9551F7E89483
:10223000EFE0FF2782910ED0EB30E0F71EF06894BC
:102240008A2D0CD088278D93EF90DF90CF90DF916F
:10225000CF910895982F829501D0892F8F70805D3E
:1022600026F0803309F4089568948D930895F999C0
:10227000FECFE1BDF2BD3196089591E001C092E03C
:102280007B3751F47FB7F894F2DF8D9180BDFA9AD5
:10229000F99A9A95C9F77FBF7727089591E001C011
:1022A00092E0E5DFF89A80B58D939A95D1F708957D
:1022B000FF93881BF9E0001FFA9511F4FF91089530
:1022C000881F841B18F4840F8894F5CF0894F3CFEB
:1022D000200047617A206E61207A65726F210000CC
:1022E0004D6F6E69746F72004B616C6962726163ED
:1022F0006A61000057797A6572756A207472796D27
:102300006572790077796368796C206472617A6BA1
:1023100069002E00284329273035205A2E4269674C
:10232000616A000020302E38352E00005620202013
:1023300000003A0030005779626F72206D6F64655B
:102340006C7500004E617A7761206D6F64656C7505
:1023500000004D696B736572000044656C74610028
:102360004D6F74796C656B004E6965207779627288
:10237000616E79004F6477726F636F6E65004E69AE
:10238000650054616B005A65726F00004D696E699B
:102390006D756D006D616B73696D756D00004E69D3
:1023A000656C696E696F776F00002C0053657277FA
:1023B00069730000416C61726D206261742E0000CF
:1023C0004C6F746B69004B696572756E656B0000CC
:0E23D0005779736F6B6F7363000047617A007B
:00000001FF
